:10000000CD2883120313A5002508A800F930840029
:100010000000840B082883120313A80B0628831200
:100020000313A501203083120313250203182E2881
:1000300005140000000000000000000000000000A7
:10004000000000000000000000000510000000009B
:100050000000000000000000A50A1228831203130C
:10006000A501203083120313250203184D28000038
:100070000000000000000000000000000000000080
:100080000000000000000000000000000000000070
:10009000000000000000A50A3128080083120313A5
:1000A000A501203083120313250203186D280000D8
:1000B0000000000000000000000000000000000040
:1000C0000000000000000000000000000000000030
:1000D000000000000000A50A512883120313A501A7
:1000E000203083120313250203188C280514000006
:1000F0000000000000000000000000000000000000
:1001000000000000000005100000000000000000DA
:1001100000000000A50A702808004E204E2083121F
:100120000313A608031D96280F2097284E20103091
:1001300083120313A300A4010530831203132402C6
:100140000318AF281D3023050319A8284E20A9281D
:100150000F20031083120313A30CA40A9C28203041
:1001600083120313A300A401063083120313240295
:100170000318C82823082705003A0319C1284E2070
:10018000C2280F20031083120313A30CA40AB4285F
:100190008312031305107130012864008130831627
:1001A00003138100073083129F0083168501F0300E
:1001B0008600F030831286008501A901AA018B1503
:1001C0000B1063000000403083120313A7008B1153
:1001D0000B10061AED28A701802183120313861A3B
:1001E000F4280430A700802183120313061BFB2888
:1001F0000830A700802183120313861B02290C30CC
:10020000A7008021083083120313270203183D2919
:100210000130A100270803191429A3000310831239
:100220000313A10DA30B0E29831203132108290523
:10023000003A03191F292109A905A60125298312BE
:1002400003132108A9040130A60083120313A0019F
:1002500083120313A008031D32298D208312031378
:10026000A00A2829F030831203130605A1002108F3
:10027000F03A031D32293230012008308312031373
:100280002702031C7F291030270203187F2908301A
:100290002702A2000130A100220803195629A30059
:1002A000031083120313A10DA30B50298312031310
:1002B00021082A05003A031961292109AA05A60186
:1002C0006729831203132108AA040130A6008312B0
:1002D0000313A00183120313A008031D74298D20AA
:1002E00083120313A00A6A29F03083120313060550
:1002F000A1002108F03A031D742932300120DF28C3
:10030000013083120313A500A301043083120313E9
:10031000230203189E2925088600F0300605A40054
:10032000F03086002408F03A031D97290800831254
:100330000313A70A0310A50DA30A85290800FF3F90
:10034000FF3FFF3FFF3FFF3FFF3FFF3FFF3FFF3FBD
:10035000FF3FFF3FFF3FFF3FFF3FFF3FFF3FFF3FAD
:10036000FF3FFF3FFF3FFF3FFF3FFF3FFF3FFF3F9D
:10037000FF3FFF3FFF3FFF3FFF3FFF3FFF3FFF3F8D
:02400E00213F50
:10420000FF00FF00FF00FF00FF00FF00FF00FF00B6
:10421000FF00FF00FF00FF00FF00FF00FF00FF00A6
:10422000FF00FF00FF00FF00FF00FF00FF00FF0096
:10423000FF00FF00FF00FF00FF00FF00FF00FF0086
:10424000FF00FF00FF00FF00FF00FF00FF00FF0076
:10425000FF00FF00FF00FF00FF00FF00FF00FF0066
:10426000FF00FF00FF00FF00FF00FF00FF00FF0056
:10427000FF00FF00FF00FF00FF00FF00FF00FF0046
:10428000FF00FF00FF00FF00FF00FF00FF00FF0036
:10429000FF00FF00FF00FF00FF00FF00FF00FF0026
:1042A000FF00FF00FF00FF00FF00FF00FF00FF0016
:1042B000FF00FF00FF00FF00FF00FF00FF00FF0006
:1042C000FF00FF00FF00FF00FF00FF00FF00FF00F6
:1042D000FF00FF00FF00FF00FF00FF00FF00FF00E6
:1042E000FF00FF00FF00FF00FF00FF00FF00FF00D6
:1042F000FF00FF00FF00FF00FF00FF00FF00FF00C6
:00000001FF
